:1000000019C233C232C231C230C22FC22EC22DC277
:100010002CC22BC22AC229C228C260C226C225C253
:1000200024C223C222C221C220C21FC21EC21DC2BC
:100030001CC21BC2808386898C8F9295989C9FA23C
:10004000A5A8ABAEB0B3B6B9BCBFC1C4C7C9CCCE0E
:10005000D1D3D5D8DADCDEE0E2E4E6E8EAECEDEF95
:10006000F0F2F3F5F6F7F8F9FAFBFCFCFDFEFEFF03
:10007000FFFFFFFFFFFFFFFFFFFFFEFEFDFCFCFB9E
:10008000FAF9F8F7F6F5F3F2F0EFEDECEAE8E6E46A
:10009000E2E0DEDCDAD8D5D3D1CECCC9C7C4C1BF4B
:1000A000BCB9B6B3B0AEABA8A5A29F9C9895928FF1
:1000B0008C898683807C797673706D6A6763605DF6
:1000C0005A5754514F4C494643403E3B38363331E2
:1000D0002E2C2A272523211F1D1B1917151312103B
:1000E0000F0D0C0A090807060504030302010100AD
:1000F00000000000000000000000010102030304F2
:1001000005060708090A0C0D0F1012131517191B05
:100110001D1F212325272A2C2E313336383B3E4004
:100120004346494C4F5154575A5D6063676A6D703E
:100130007376797C030303030303030303030303BD
:10014000030303030303030303030303030303037F
:100150000303030303030303030303030303000075
:1001600000000F0F0F0F0303030303030303030335
:100170000303030303030303030303030303000055
:1001800000000F0F0F0F0F0F0303030303030303FD
:10019000030303030303030303030303030F000029
:1001A00000000F0F0F0F0F0F0F0F030303030303C5
:1001B000030303030303030303030303030F000009
:1001C00000000F0F0F0F0F0F0F0F030303030303A5
:1001D0000303030303030303030303030F0F0000DD
:1001E00000003F3F3F3F3F3F3F0F0F030303030329
:1001F0000303030303030303030303030F0F0000BD
:1002000000003F3F3F3F3F3F3F0F0F030303030308
:1002100003030303030303030303030F0F0F000090
:1002200000003F3F3F3F3F3F3F0F0F0F03030303DC
:1002300003030303030303030303030F0F0F000070
:1002400000003F3F3F3F3F3F3F0F0F0F03030303BC
:1002500003030303030303030303030F0F0F000050
:1002600000000000003F3F3F3F0F0F0F0303030359
:1002700003030303030303030303030F0F0F000030
:1002800000000000003F3F3F3F0F0F0F0303030339
:100290000303030303030303030303030F0F00001C
:1002A00000000000003F3F3F3F0F0F030303030325
:1002B0000303030303030303030303030F0F0000FC
:1002C00000000000003F3F3F3F0F0F030303030305
:1002D000030303030303030303030303030F0F0FCA
:1002E0000F0F0F0F0F3F3F3F3F0F030303030303A6
:1002F000030303030303030303030303030F0F0FAA
:100300000F0F0F0F0F3F3F3F3F0F03030303030385
:100310000303030303030303030303030303030FA1
:100320000F0F0F0F0F3F3F3F3F0303030303030371
:10033000030303030303030303030303030303038D
:10034000030F0F0F0F3F3F3F3F030303030303035D
:10035000030303030303030303030303030303036D
:10036000030303030303030303030303030303035D
:10037000030303030000030300000000000000006B
:100380000000000000000003030000000000000067
:10039000030000003F000300003F00003F003F005B
:1003A000003F3F003F3F000000003F0000003F00D3
:1003B00000003F3F3F0003003F003F003F003F0081
:1003C0003F0000003F003F00003F003F003F003F74
:1003D000003F00002A0003002A2A2A00002A000009
:1003E0002A2A00002A2A0000002A002A002A002ABD
:1003F000002A2A002A0000002A002A00002A000001
:100400002A0000002A002A00002A002A002A002AC6
:10041000002A000000151500150015000015000049
:100420000015150015001500000015000015001539
:100430000000151511241FBECFEFD4E0DEBFCDBFE5
:1004400011E0A0E0B1E0E6E9F6E002C005900D920F
:10045000A830B107D9F714E0A8E0B1E001C01D92BF
:10046000AC30B107E1F7A0D014C1CACD84B1866029
:1004700084B98FE387B915B818B8E0E8F0E080E2F6
:100480008083808182608083A1E8B0E088E18C93E2
:100490008FE092E090938700809386008FE390E056
:1004A00090938B0080938A0080818068808380E1B4
:1004B00092E0909389008093880010920904109232
:1004C000080488E091E090930B0480930A048C91D7
:1004D00081608C9381E080936F0008950F920FB636
:1004E0000F928F939F93FF93EF93809108049091C5
:1004F0000904039731F4E0E8F0E08081806C8083A8
:1005000034C0489790F18835F2E09F0770F51F924C
:100510002F931F930F93E0910A04F0910B0409E2CB
:10052000809F812D909F800D8695869500E2809F0B
:10053000E00DF11D0DE510918400011B0350F4F74F
:10054000039504F4039504F410E2219128B921E005
:100550002A95F1F710FD0000000000001A95A9F798
:1005600018B90F911F912F911F90809108049091BD
:1005700009040196909309048093080484379240FB
:1005800059F411241092090410920804E0E8F0E0F4
:10059000808180688F7B8083EF91FF919F918F9105
:1005A0000F900FBE0F901895CF93DF93CDB7DEB7A6
:1005B00028970FB6F894DEBF0FBECDBF88E0E0E00D
:1005C000F1E0DE01119601900D928A95E1F74EDF80
:1005D00040E053E064E371E088E091E051D078942A
:1005E000D12CAAE0CA2E60E270E02D2D30E040E070
:1005F00050E0890180E090E0F901FF27EC5CFF4FBB
:10060000E4915801AE0EB11CCA9CD001CB9CB00D38
:1006100011247C01E40EF51EF701EC5CFE4FE49121
:10062000E330F9F4FB01E81BF90BAA2EE89FA00CBC
:100630001124EA2DF0E0EC5CFF4FB490F701E85F85
:10064000FE4F7F01EB2DE295E695E770AA24A39477
:10065000B12CAC0EBD1EAE0EB11CF501B080F70181
:10066000B082019680329105A1F6405E5F4F2F5F08
:100670003F4F4115F3E05F0709F0BCCFD394B5CFEE
:10068000FB01DC0102C005900D9241505040D8F7AB
:060690000895F894FFCF6D
:08069600010203132333373B7B
:00000001FF
